:1000000012C02AC029C028C027C026C025C024C0CD
:1000100023C022C021C020C01FC01EC01DC01CC0E4
:100020001BC01AC019C011241FBECFEDCDBF10E0F8
:10003000A0E6B0E0E4E6F7E003C0C89531960D9283
:10004000A036B107D1F710E0A0E6B0E001C01D92E4
:10005000A33AB107E1F7DCC0D3CF81E45DD286E5F6
:100060005BD282E559D280E257D289E455D283E54A
:1000700053D280E551D208950F931F93CF93182F39
:100080004FD2082F4DD2C82F802FF9D18C2FF7D106
:1000900047D2F5D1112369F043D20C3A59F4C03A52
:1000A00011F0C03E11F48FEF05C0C83A19F489E48D
:1000B00001C0812FE4D130D285E090E075D18DE090
:1000C0002BD2CF911F910F910895BA9A82E480BFED
:1000D00081E083BF86BF12BE0895DF92EF92FF9248
:1000E0000F931F93CF93DF93E82EF92ED62E20E0A7
:1000F00030E0D32FC22FC05ADF4F022F132F0F5FD4
:100100001F4F2E153F0510F40BD201C08FEF8883CF
:10011000312F202F0034110560F320E030E0809172
:10012000A2008A3319F0932F822F3CC00091A000C7
:100130001091A10086E4D81699F5CFE5D0E080E4CF
:100140009ED18091A1009BD18091A00098D1219651
:10015000899195D188E493D18091A10090D180912B
:10016000A0008DD188818BD18091A0009091A100B9
:1001700001969093A1008093A0008EEF9FEFE80E70
:10018000F91EE114F104D9F68CE479D1812F992775
:1001900076D1802F74D180E072D185E090E004D1D7
:1001A0008DE090E0DF91CF911F910F91FF90EF9044
:1001B000DF900895CF93DF93D92FC82F663429F5A8
:1001C0008091A2008A3309F580E259D18091A10083
:1001D00056D18091A00053D18FEF51D19DD188E2AB
:1001E0004ED18091A1004BD18091A00048D18FEFDA
:1001F00046D192D18091A0009091A1000196909358
:10020000A1008093A0002297F9F6DF91CF91089585
:10021000CFEDD0E0DEBFCDBFF89457DFB898C09ADD
:100220000000B099FFCF21D108D160E08BE090E0D1
:1002300068D1B99AC19A74D1813611F489E5B2C0F6
:10024000813489F46DD199279093A1008093A00007
:10025000182F002765D19927082B192B1093A1007F
:100260000093A0003CC0823631F489E555D180E08E
:1002700053D180E497C0823471F452D19927182F5A
:1002800000274ED19927082B192B4AD1682F912F7F
:10029000802F23DF87C0873671F442D19927182F2A
:1002A00000273ED19927082B192B3AD1682F912F7F
:1002B000802F80DFC0CF853631F48091A2008A3351
:1002C00071F413D10CC0853461F4BCD088E190E0A6
:1002D00028E00FB6F894A89581BD0FBE21BD8DE032
:1002E00061C0803511F4E2D0FACF8C3411F4F4D02F
:1002F000F6CF803711F483E555C0823711F48FEFC4
:1003000051C08C3611F40CD1EACF843721F48AE342
:1003100003D180E047C0883729F402D1823029F424
:10032000C198DDCF893719F4FBD0C19AD8CF843575
:1003300021F4F6D08093A200D2CF833511F48DDE64
:100340007ACF863521F480E3E7D082E32BC0833770
:1003500099F48091A2008A3309F06DCF03E0015037
:1003600080E38DD080E08BD0802F89D08FEF87D035
:10037000D3D00023A1F75FCF8D3439F488B392E056
:10038000892788BB84E7C8D0AACF8A3311F480E0DC
:1003900003C08E3219F481E06FDE4DCF8B3109F44A
:1003A0004ACF8FE3B9D047CFEF92FF920F931F93BD
:1003B000082F192F802F912FAA2797FDA095BA2FCC
:1003C000682F792F8A2F9B2F10D117FF05C020E0AF
:1003D00030E040E857E4AAD026E636E646E654E4A4
:1003E00070D1E62EF72E082F192F20E030E040E8DC
:1003F0005FE305D188231CF481E090E017C020E082
:100400003FEF4FE757E4912F802F7F2D6E2DFAD0CD
:1004100018161CF480E090E009C0912F802F7F2DEA
:100420006E2DC6D0B92FA82F972F862F0197F1F7E1
:100430001F910F91FF90EF900895C49885E190E08F
:10044000B3DF0895C49A85E190E0AEDF0895FADF46
:10045000F4DF089589E00000815087FFFCCF089504
:10046000C79AF8DFC798F6DF0895BC9A0895C79A2F
:1004700087B3806A87BBF9DFBE98F2DF08950F93D8
:100480001F93CF93082F10E0C0E8802F8C2311F02A
:10049000C59A01C0C598B6991C0FE2DFC695A9F7A9
:1004A000812F9927CF911F910F910895CF93DFDF6F
:1004B000CEDFC0E08CEAE3DF83E5E1DF8FEFDFDF53
:1004C000833511F4C1E401C0C2DF80E0D8DFCF5F23
:1004D000C03480F3CF910895BADF8FE597B39823A6
:1004E00097BB98B3982398BB08958CEAC8DF80E83F
:1004F000C6DF80E0C4DF80E0C2DF8AE090E054DF46
:100500000895282F392F832F992782B929B988E197
:100510008AB986E083B908955D9BFECF8CB90895B2
:100520005F9BFECF8CB1992708955058192EA6D005
:1005300001D08CC0BA176207730784079507B1F121
:1005400088F40EF410940B2EBA2FA02D062E622FD5
:10055000202D072E732F302D082E842F402D092E8D
:10056000952F502DFF275523B9F0591B49F0573EC1
:1005700098F0469537952795A795F0405395C9F77C
:1005800076F0BA0F621F731F841F30F4879577953A
:100590006795B795F040939517FA0F2E0895BF1BF6
:1005A000BB27BA0B620B730B840BF6CFDEF683C04E
:1005B00097FB70D09F3738F0FEE9F91B982F872FF3
:1005C000762F6B2F05C074C09695879577956795A4
:1005D000F150D0F73EF490958095709561957F4FDE
:1005E0008F4F9F4F0895E89403C097FB0EF4F3DFFD
:1005F000B62F672F782F892F9EE9002427C00ED0B1
:100600005EF004C00BD026F001C008D019F020F431
:100610008FEF089580E0089581E0089597FB092EFB
:10062000052600F868942DD0E89407FC07C06217EF
:1006300073078407950721F008F4009407949894B1
:1006400008959A95BB0F661F771F881F1124992361
:10065000A1F08823B2F79F3F59F0BB0F48F421F473
:10066000002011F460FF04C06F5F7F4F8F4F9F4FDA
:10067000881F9795879597F908951AC0052E092622
:1006800007FA440F551F5F3F79F0AA27A51708F016
:1006900051E04795880F991F9F3F31F0BB27B9174D
:1006A00008F091E0879508959F919F91112457C07C
:1006B00066277727882799270895592F482F372F9E
:1006C000262FDCDF01D0C2CF992339F0552329F042
:1006D0009F575F57950F13F4CAF1EDCF91589F3F85
:1006E000E1F3A62F00241124BB2766275527F8E045
:1006F000A69520F4020E131EB41F651F220F331F90
:10070000441F551FFA95A1F7F8E0E72F7727F8E087
:10071000E69520F4130EB41F651F7A1F330F441F94
:10072000551FAA1FFA95A1F7F82F8827F69520F4F0
:10073000B40F651F7A1F8E1F440F551FAA1FEE1F8F
:10074000FF23A1F788231AF4939539F408C0000C0D
:10075000111CBB1F661F771F881F012808959FEF7C
:0407600080EC08958C
:00000001FF
